:100000000C9462060C948A060C948A060C948A0658
:100010000C948A060C948A060C948A060C948A0620
:100020000C948A060C948A060C948A060C948A0610
:100030000C948A060C948A060C948A060C948A0600
:100040000C9494080C948A060C948A060C948A06E4
:100050000C948A060C948A060C948A060C948A06E0
:100060000C948A060C948A06FFFEFDFCFBFAF9F854
:10007000F7F6F5F4F3F2F1F0EFEEEDECEBEBEAE985
:10008000E8E7E6E5E4E3E2E1E0E0DFDEDDDCDBDA61
:10009000D9D9D8D7D6D5D4D3D3D2D1D0CFCECECD2F
:1000A000CCCBCACAC9C8C7C6C6C5C4C3C2C2C1C0F0
:1000B000BFBFBEBDBCBCBBBAB9B9B8B7B6B6B5B4A4
:1000C000B3B3B2B1B1B0AFAEAEADACACABAAAAA94E
:1000D000A8A8A7A6A6A5A4A4A3A2A2A1A0A09F9EEB
:1000E0009E9D9D9C9B9B9A9999989897969695957D
:1000F00094939392929190908F8F8E8E8D8C8C8B07
:100100008B8A8A8988888787868685858484838385
:1001100082818180807F7F7E7E7D7D7C7C7B7B7AFF
:100120007A7979787877777676757575747473736C
:100130007272717170706F6F6F6E6E6D6D6C6C6BD3
:100140006B6B6A6A69696868686767666665656532
:100150006464636363626261616160605F5F5F5E8C
:100160005E5D5D5D5C5C5C5B5B5A5A5A59595958DF
:10017000585857575656565555555454545353532B
:100180005252525151515050504F4F4F4E4E4E4D72
:100190004D4D4C4C4C4B4B4B4A4A4A4A49494948B5
:1001A00048484747474746464645454545444444F1
:1001B0004343434342424241414141404040403F2A
:1001C0003F3F3E3E3E3E3D3D3D3D3C3C3C3C3B3B5F
:1001D0003B3B3A3A3A3A393939393838383838378E
:1001E00037373736363636353535353534343434B9
:1001F00033333333333232323231313131313030E3
:100200003030302F2F2F2F2F2E2E2E2E2E2D2D2D06
:100210002D2D2C2C2C2C2C2B2B2B2B2B2B2A2A2A28
:100220002A2A292929292929282828282828272746
:100230002727272626262626262525252525252562
:10024000242424242424232323232323222222227C
:100250002222222121212121212120202020202091
:10026000201F1F1F1F1F1F1F1E1E1E1E1E1E1E1DA6
:100270001D1D1D1D1D1D1D1C1C1C1C1C1C1C1C1BB8
:100280001B1B1B1B1B1B1B1A1A1A1A1A1A1A1A19C8
:1002900019191919191919191818181818181818D6
:1002A00017171717171717171717161616161616E4
:1002B00016161615151515151515151515141414EE
:1002C00014141414141414131313131313131313F7
:1002D00013131212121212121212121212121111FE
:1002E0001111111111111111111010101010101005
:1002F0001010101010100F0F0F0F0F0F0F0F0F0F08
:100300000F0F0F0E0E0E0E0E0E0E0E0E0E0E0E0E0A
:100310000D0D0D0D0D0D0D0D0D0D0D0D0D0D0D0C0E
:100320000C0C0C0C0C0C0C0C0C0C0C0C0C0C0B0B0F
:100330000B0B0B0B0B0B0B0B0B0B0B0B0B0B0A0A0F
:100340000A0A0A0A0A0A0A0A0A0A0A0A0A0A0A0A0D
:10035000090909090909090909090909090909090D
:10036000090908080808080808080808080808080B
:100370000808080808080707070707070707070707
:100380000707070707070707070707070606060601
:1003900006060606060606060606060606060606FD
:1003A00006060606050505050505050505050505F9
:1003B00005050505050505050505050505050404EF
:1003C00004040404040404040404040404040404ED
:1003D00004040404040404040404040303030303E2
:1003E00003030303030303030303030303030303DD
:1003F00003030303030303030303030302020202D1
:1004000002020202020202020202020202020202CC
:1004100002020202020202020202020202020202BC
:1004200002020101010101010101010101010101BA
:1004300001010101010101010101010101010101AC
:10044000010101010101010101010101010101009D
:10045000000000000000000000000000000000009C
:100460000000000000000000000005000A000F006E
:10047000140019001E00230027002C003100360054
:100480003B003F00440049004D00520057005B0014
:100490006000640069006D00720076007B007F00E0
:1004A000840088008C009100950099009E00A200B5
:1004B000A600AA00AE00B300B700BB00BF00C30097
:1004C000C700CB00CF00D300D700DB00DF00E30084
:1004D000E700EB00EF00F300F600FA00FE00020177
:1004E000060109010D011101140118011C011F0170
:1004F000230127012A012E013101350138013C0178
:100500003F01430146014A014D0150015401570189
:100510005B015E016101640168016B016E017101A3
:10052000750178017B017E018101850188018B01C4
:100530008E019101940197019A019D01A001A301EF
:10054000A601A901AC01AF01B201B501B801BB011F
:10055000BD01C001C301C601C901CB01CE01D1015A
:10056000D401D701D901DC01DF01E101E401E70198
:10057000E901EC01EF01F101F401F601F901FB01E0
:10058000FE0101020302060208020B020D020F0225
:1005900012021402170219021C021E022002230278
:1005A000250227022A022C022E02310233023502D2
:1005B00038023A023C023E02400243024502470230
:1005C00049024B024E025002520254025602580295
:1005D0005A025C025E0260026302650267026902FF
:1005E0006B026D026F02710273027502770278026C
:1005F0007A027C027E0280028202840286028802E3
:100600008A028B028D028F0291029302950296025A
:1006100098029A029C029D029F02A102A302A402D8
:10062000A602A802AA02AB02AD02AF02B002B20259
:10063000B402B502B702B902BA02BC02BD02BF02DF
:10064000C102C202C402C502C702C802CA02CC0269
:10065000CD02CF02D002D202D302D502D602D802F6
:10066000D902DB02DC02DD02DF02E002E202E30289
:10067000E502E602E702E902EA02EC02ED02EE021E
:10068000F002F102F202F402F502F602F802F902B7
:10069000FA02FC02FD02FE02FF0201030203030351
:1006A00005030603070308030A030B030C030D03EA
:1006B0000E0310031103120313031403160317038D
:1006C000180319031A031B031D031E031F03200332
:1006D00021032203230324032503270328032903DB
:1006E0002A032B032C032D032E032F033003310386
:1006F0003203330334033503360337033803390336
:100700003A033B033C033D033E033F0340034103E5
:100710004203430344034503460347034803490395
:100720004A034B034B034C034D034E034F0350034B
:100730005103520353035303540355035603570302
:100740005803590359035A035B035C035D035E03BB
:100750005E035F0360036103620363036303640377
:100760006503660366036703680369036A036A0334
:100770006B036C036D036D036E036F0370037003F3
:1007800071037203720373037403750375037603B5
:10079000770377037803790379037A037B037C0378
:1007A0007C037D037E037E037F037F03800381033D
:1007B0008103820383038303840385038503860304
:1007C000870387038803880389038A038A038B03CB
:1007D0008B038C038D038D038E038E038F03900395
:1007E0009003910391039203920393039403940360
:1007F000950395039603960397039703980398032D
:10080000990399039A039B039B039C039C039D03F9
:100810009D039E039E039F039F03A003A003A103C8
:10082000A103A203A203A303A303A403A403A50398
:10083000A503A503A603A603A703A703A803A8036C
:10084000A903A903AA03AA03AB03AB03AB03AC033D
:10085000AC03AD03AD03AE03AE03AE03AF03AF0312
:10086000B003B003B103B103B103B203B203B303E6
:10087000B303B303B403B403B503B503B503B603BD
:10088000B603B703B703B703B803B803B903B90393
:10089000B903BA03BA03BA03BB03BB03BB03BC036C
:1008A000BC03BD03BD03BD03BE03BE03BE03BF0344
:1008B000BF03BF03C003C003C003C103C103C1031F
:1008C000C203C203C203C303C303C303C403C403F9
:1008D000C403C503C503C503C603C603C603C703D4
:1008E000C703C703C703C803C803C803C903C903B1
:1008F000C903CA03CA03CA03CA03CB03CB03CB038E
:10090000CC03CC03CC03CC03CD03CD03CD03CE036A
:10091000CE03CE03CE03CF03CF03CF03CF03D00349
:10092000D003D003D103D103D103D103D203D20327
:10093000D203D203D303D303D303D303D403D40307
:10094000D403D403D503D503D503D503D503D603E8
:10095000D603D603D603D703D703D703D703D803C9
:10096000D803D803D803D803D903D903D903D903AB
:10097000DA03DA03DA03DA03DA03DB03DB03DB038C
:10098000DB03DB03DC03DC03DC03DC03DC03DD0370
:10099000DD03DD03DD03DD03DE03DE03DE03DE0353
:1009A000DE03DF03DF03DF03DF03DF03E003E00336
:1009B000E003E003E003E103E103E103E103E1031A
:1009C000E103E203E203E203E203E203E203E303FF
:1009D000E303E303E303E303E403E403E403E403E3
:1009E000E403E403E503E503E503E503E503E503C9
:1009F000E503E603E603E603E603E603E603E703AF
:100A0000E703E703E703E703E703E703E803E80394
:100A1000E803E803E803E803E803E903E903E9037B
:100A2000E903E903E903E903EA03EA03EA03EA0362
:100A3000EA03EA03EA03EB03EB03EB03EB03EB0349
:100A4000EB03EB03EB03EC03EC03EC03EC03EC0331
:100A5000EC03EC03ED03ED03ED03ED03ED03ED0318
:100A6000ED03ED03ED03EE03EE03EE03EE03EE0301
:100A7000EE03EE03EE03EF03EF03EF03EF03EF03E9
:100A8000EF03EF03EF03EF03F003F003F003F003D2
:100A9000F003F003F003F003F003F103F103F103BB
:100AA000F103F103F103F103F103F103F103F203A5
:100AB000F203F203F203F203F203F203F203F2038E
:100AC000F203F203F303F303F303F303F303F30378
:100AD000F303F303F303F303F403F403F403F40362
:100AE000F403F403F403F403F403F403F403F4034E
:100AF000F503F503F503F503F503F503F503F50336
:100B0000F503F503F503F503F603F603F603F60321
:100B1000F603F603F603F603F603F603F603F6030D
:100B2000F603F703F703F703F703F703F703F703F6
:100B3000F703F703F703F703F703F703F803F803E3
:100B4000F803F803F803F803F803F803F803F803CD
:100B5000F803F803F803F803F803F903F903F903BA
:100B6000F903F903F903F903F903F903F903F903A5
:100B7000F903F903F903F903F903FA03FA03FA0392
:100B8000FA03FA03FA03FA03FA03FA03FA03FA037D
:100B9000FA03FA03FA03FA03FA03FA03FB03FB036B
:100BA000FB03FB03FB03FB03FB03FB03FB03FB0355
:100BB000FB03FB03FB03FB03FB03FB03FB03FB0345
:100BC000FB03FC03FC03FC03FC03FC03FC03FC032E
:100BD000FC03FC03FC03FC03FC03FC03FC03FC031D
:100BE000FC03FC03FC03FC03FC03FD03FD03FD030A
:100BF000FD03FD03FD03FD03FD03FD03FD03FD03F5
:100C0000FD03FD03FD03FD03FD03FD03FD03FD03E4
:100C1000FD03FD03FD03FD03FE03FE03FE03FE03D0
:100C2000FE03FE03FE03FE03FE03FE03FE03FE03BC
:100C3000FE03FE03FE03FE03FE03FE03FE03FE03AC
:100C4000FE03FE03FE03FE03FE03FE03FF03FF039A
:100C5000FF03FF03FF03FF03FF03FF03FF03FF0384
:100C6000FF03FF03FF03FF03000000002400270031
:100C70002A0000000000250028002B0000000000D2
:100C800023002600290004040404040404040202CE
:100C900002020202030303030303010204081020FB
:100CA0004080010204081020010204081020000006
:100CB000000800020100000304070000000000001B
:100CC00000002A0B11241FBECFEFD8E0DEBFCDBF3E
:100CD00011E0A0E0B1E0EAE7FDE102C005900D926D
:100CE000A832B107D9F721E0A8E2B1E001C01D9216
:100CF000AF34B207E1F716E0C2E6D6E004C02197B0
:100D0000FE010E94B50EC136D107C9F70E94DE0868
:100D10000C94BB0E0C940000833081F028F48130D9
:100D200099F08230A9F008958730A9F08830C9F091
:100D30008430B1F4809180008F7D03C08091800069
:100D40008F7780938000089584B58F7784BD089550
:100D500084B58F7DFBCF8091B0008F778093B000FA
:100D600008958091B0008F7DF9CFCF93DF93282F26
:100D700030E0F901E255F34F8491F901E656F34F63
:100D8000D491F901EA57F34FC491CC23A1F081111A
:100D90000E948C06EC2FF0E0EE0FFF1FE458F34F9B
:100DA000A591B491EC91ED2381E090E009F480E00D
:100DB000DF91CF91089580E090E0FACF1F93CF9319
:100DC000DF93282F30E0F901E255F34F8491F901C8
:100DD000E656F34FD491F901EA57F34FC491CC236F
:100DE000A9F0162F81110E948C06EC2FF0E0EE0F77
:100DF000FF1FEE58F34FA591B4918FB7F894EC9183
:100E0000111108C0D095DE23DC938FBFDF91CF9105
:100E10001F910895DE2BF8CFCF93DF9390E0FC0174
:100E2000E656F34F24918A57934FFC01849188230F
:100E3000C9F090E0880F991FFC01E859F34FA59184
:100E4000B491FC01EE58F34FC591D49161110DC0DE
:100E50009FB7F8948C91209582238C9388812823C6
:100E600028839FBFDF91CF910895623051F49FB7DF
:100E7000F8943C91822F809583238C93E8812E2BCC
:100E8000EFCF8FB7F894EC912E2B2C938FBFEACF36
:100E90001F93CF93DF93182FEB0161E00E940C07A3
:100EA000209739F460E0812FDF91CF911F910C944E
:100EB000DE06CF3FD10511F461E0F5CFE12FF0E080
:100EC000E255F34FE491E33031F140F4E130B1F019
:100ED000E230E1F0C038D1057CF7E4CFE73029F10A
:100EE000E83059F1E430B1F780918000806280935E
:100EF0008000D0938B00C0938A0004C084B58068C2
:100F000084BDC7BDDF91CF911F91089584B58062E4
:100F100084BDC8BDF7CF8091800080688093800039
:100F2000D0938900C0938800EDCF8091B000806895
:100F30008093B000C093B300E5CF8091B000806291
:100F40008093B000C093B400DDCF8E508064809356
:100F50007C0080917A00806480937A0080917A008E
:100F600086FDFCCF80917800909179000895CF9212
:100F7000DF92EF92FF92CF93DF93EC018885998502
:100F8000C880D980EA80FB808130910509F078C063
:100F9000C701B6010E94330DFB01E859FF4FE491F0
:100FA0002E813F81032E000C440B550B2F5F31091E
:100FB00041095109AE2FB0E00E940B0C2FEF30E039
:100FC00040E050E00E94EC0B21503F4F4F4F5F4FED
:100FD0003D832C836D857E85072E000C880B990B35
:100FE0000E946B0D2DEC3CEC4CEC5CE30E94200E5F
:100FF000A70196010E94500C688379838A839B83A2
:10100000C880D980EA80FB8020E030E040E854E4EA
:10101000C701B6010E941B0E181674F420E030E0E0
:1010200040E055E4C701B6010E94BC0C87FF04C034
:1010300082E090E09987888720E030E040E055E446
:10104000C701B6010E941B0E87FD08C018821982D5
:101050001A821B821986188681E08A878A858823EE
:1010600041F08B859C8501968B309105DCF49C8743
:101070008B87DF91CF91FF90EF90DF90CF90089515
:10108000029709F0BDCFC701B6010E94330DFB01E5
:10109000F450E859FF4FE491F0E0FD83EC836F8555
:1010A00078899ACF1C861B861A86E3CF8F929F92EF
:1010B000AF92BF92CF92DF92EF92FF924A015B0113
:1010C000BC01990F880B990B0E946B0D6B017C0181
:1010D0000E94940B20ED37E040E050E00E94EC0BC2
:1010E000685E7340810991090E946B0D20E030E039
:1010F0004AE754E40E94C10CA70196010E94200E09
:10110000A50194010E94200EA70196010E94500C97
:101110000E94330DCB01FF90EF90DF90CF90BF90F6
:10112000AF909F908F9008951F920F920FB60F92DD
:1011300011242F933F938F939F93AF93BF938091ED
:101140004B0190914C01A0914D01B0914E01309115
:101150004A0123E0230F2D3758F50196A11DB11D3B
:1011600020934A0180934B0190934C01A0934D0131
:10117000B0934E018091460190914701A0914801A2
:10118000B09149010196A11DB11D80934601909334
:101190004701A0934801B0934901BF91AF919F913E
:1011A0008F913F912F910F900FBE0F901F90189528
:1011B00026E8230F0296A11DB11DD2CFCF93DF9356
:1011C00000D000D0CDB7DEB7789484B5826084BDFE
:1011D00084B5816084BD85B5826085BD85B581603B
:1011E00085BD80916E00816080936E0010928100B9
:1011F0008091810082608093810080918100816074
:101200008093810080918000816080938000809134
:10121000B10084608093B1008091B00081608093C0
:10122000B00080917A00846080937A0080917A0087
:10123000826080937A0080917A00816080937A0046
:1012400080917A00806880937A001092C10062E0F9
:1012500084E00E940C0760E081E10E940C0760E0DE
:101260008AE00E940C0761E083E00E940C0761E0C5
:1012700089E00E940C0761E08BE00E940C0783E28A
:101280008093B00081E08093B10082E88093800079
:1012900089E1809381008FEF90E0909387008093A5
:1012A00086008FB7F894C0904B01D0904C01E0902D
:1012B0004D01F0904E018FBFC0924201D092430188
:1012C000E0924401F09245018EE00E94A5078C0156
:1012D0008FE00E94A5079C838B8380E10E94A50775
:1012E000BC01F801EE0FFF1FE859FB4F8591949167
:1012F000212C24E0322E281A390A30924101209202
:101300004001EB81FC81EE0FFF1FE859FB4F8591F7
:10131000949120E034E0281B390B3A8329833093E1
:101320003F0120933E01072E000C880B990B0E9471
:101330006B0D20E030EC4FE754E40E94C10C4B01F0
:101340005C01B801110F880B990B0E946B0D20E016
:1013500030EC4FE754E40E94C10C9B01AC0160E00B
:1013600070E080E89FE30E944F0C2AE939E949E1E7
:101370005FE30E94200E2DEC3CEC4CE45EE30E9407
:10138000500CA50194010E94200E2B013C012B81E1
:101390003C81B901330F880B990B0E946B0D20E043
:1013A00030EC4FE754E40E94C10C9B01AC0160E0BB
:1013B00070E080E89FE30E944F0C2AE939E949E197
:1013C0005FE30E94200E2DEC3CEC4CE45EE30E94B7
:1013D000500CA50194010E94200E4B015C0184E099
:1013E0000E94B50610923C0110923D0190913B0184
:1013F000891751F080933B01C0923601D09237019A
:10140000E0923801F09239018091360190913701D4
:10141000A0913801B0913901C81AD90AEA0AFB0A29
:101420008091320190913301A0913401B091350146
:101430008C159D05AE05BF05B0F490913A018091E1
:101440003B01981781F080933A01911103C021E08C
:10145000813009F020E020933C01913009F48111A2
:1014600090E090933D0181E10E94B50620912F010B
:10147000211103C091E0813009F090E09093300198
:10148000213011F491E0811190E09093310180932B
:101490002F018AE00E94B50620912C01211103C082
:1014A00091E0813009F090E090932D01213019F402
:1014B00031E03B8381111B824B8140932E0180934D
:1014C0002C0180913D01811104C08091310188235C
:1014D00081F180911A0190911B01029709F0B4C02B
:1014E0008091160190911701909319018093180132
:1014F00081E090E090931B0180931A0110921201F9
:10150000109213011092140110921501B301A2015F
:10151000C1010E9456089093200180931F01B501DC
:10152000A40189819A810E94560890932201809398
:1015300021019B819923D1F120913E0130913F01FE
:101540003A832983809140019091410120910801C3
:10155000309109012230310509F079C02091040150
:1015600030910501309307012093060121E030E01E
:10157000309309012093080110920001109201019B
:101580001092020110920301B301A2010E945608B9
:1015900090930E0180930D01B501A40189819A8178
:1015A0000E9456089093100180930F018091420190
:1015B00090914301A0914401B091450140912801CF
:1015C0005091290160912A0170912B018417950790
:1015D000A607B70789F18093280190932901A0936A
:1015E0002A01B0932B0182E191E00E94B70780E0CD
:1015F00091E00E94B70760911601709117018091E8
:1016000023010E944807209116013091170140EAFA
:10161000429FC001439F900D11246FEF70E00E9424
:101620008D0E83E00E9448076091040170910501CE
:10163000809111010E94480780E090E0892B09F415
:1016400030CE0E9400002DCE90E080E04DCF30E003
:1016500020E088CFE2E3F1E082E390E0A0E0B0E0B8
:1016600080839183A283B3831482158216821782AA
:1016700081E08087818712861386EFE2F1E0808324
:1016800011821282ECE2F1E08083118212820895CD
:101690008F929F92AF92BF92CF92DF92EF92FF9282
:1016A000CF93DF93EC01688179818A819B816115F9
:1016B00071058105910521F464E279ED8BE597E0F0
:1016C0002DE133EF41E050E00E94EC0B49015A015B
:1016D0009B01AC01A7EAB1E40E940B0C6B017C01F9
:1016E000ACEEB4EFA50194010E94190CC60ED71EF2
:1016F000E81EF91EF7FE06C081E0C81AD108E1080D
:1017000080E8F80AC882D982EA82FB82C701B60162
:101710009F77DF91CF91FF90EF90DF90CF90BF90B8
:10172000AF909F908F9008958F929F92AF92BF92AB
:10173000CF92DF92EF92FF92609124017091250188
:101740008091260190912701611571058105910510
:1017500021F464E279ED8BE597E02DE133EF41E090
:1017600050E00E94EC0B49015A019B01AC01A7EA31
:10177000B1E40E940B0C6B017C01ACEEB4EFA5014F
:1017800094010E94190CC60ED71EE81EF91EF7FE22
:1017900006C081E0C81AD108E10880E8F80AC092C2
:1017A0002401D0922501E0922601F0922701C70181
:1017B000B6019F77FF90EF90DF90CF90BF90AF90F2
:1017C0009F908F90089560932401709325018093DA
:1017D0002601909327010895052E97FB1EF400948F
:1017E0000E94030C57FD07D00E941E0C07FC03D07B
:1017F0004EF40C94030C50954095309521953F4F35
:101800004F4F5F4F089590958095709561957F4FEC
:101810008F4F9F4F08950E94400CA59F900DB49F3D
:10182000900DA49F800D911D11240895B7FF0C9475
:101830000B0C0E940B0C821B930B0895A1E21A2E35
:10184000AA1BBB1BFD010DC0AA1FBB1FEE1FFF1F64
:10185000A217B307E407F50720F0A21BB30BE40BB4
:10186000F50B661F771F881F991F1A9469F76095FB
:101870007095809590959B01AC01BD01CF010895B5
:10188000A29FB001B39FC001A39F700D811D1124C1
:10189000911DB29F700D811D1124911D0895505806
:1018A000BB27AA270E94670C0C94E10D0E94D30D60
:1018B00038F00E94DA0D20F039F49F3F19F426F435
:1018C0000C94D00D0EF4E095E7FB0C94CA0DE92FB3
:1018D0000E94F20D58F3BA17620773078407950741
:1018E00020F079F4A6F50C94140E0EF4E0950B2E6E
:1018F000BA2FA02D0B01B90190010C01CA01A00162
:101900001124FF27591B99F0593F50F4503E68F1BC
:101910001A16F040A22F232F342F4427585FF3CFFD
:10192000469537952795A795F0405395C9F77EF4CE
:101930001F16BA0B620B730B840BBAF09150A1F017
:10194000FF0FBB1F661F771F881FC2F70EC0BA0F9D
:10195000621F731F841F48F4879577956795B79525
:10196000F7959E3F08F0B0CF9395880F08F0992720
:10197000EE0F9795879508950E94A60D08F481E0D3
:1019800008950E94D50C0C94E10D0E94DA0D58F0D8
:101990000E94D30D40F029F45F3F29F00C94CA0D4A
:1019A00051110C94150E0C94D00D0E94F20D68F399
:1019B0009923B1F3552391F3951B550BBB27AA2708
:1019C00062177307840738F09F5F5F4F220F331F42
:1019D000441FAA1FA9F335D00E2E3AF0E0E832D00A
:1019E00091505040E695001CCAF72BD0FE2F29D00D
:1019F000660F771F881FBB1F261737074807AB07DF
:101A0000B0E809F0BB0B802DBF01FF2793585F4F53
:101A10003AF09E3F510578F00C94CA0D0C94150EC7
:101A20005F3FE4F3983ED4F3869577956795B79535
:101A3000F7959F5FC9F7880F911D9695879597F940
:101A40000895E1E0660F771F881FBB1F62177307B9
:101A50008407BA0720F0621B730B840BBA0BEE1FCE
:101A600088F7E09508950E943A0D6894B1110C949E
:101A7000150E08950E94FA0D88F09F5798F0B92F1F
:101A80009927B751B0F0E1F0660F771F881F991FB3
:101A90001AF0BA95C9F714C0B13091F00E94140E33
:101AA000B1E008950C94140E672F782F8827B85F43
:101AB00039F0B93FCCF3869577956795B395D9F70B
:101AC0003EF490958095709561957F4F8F4F9F4F15
:101AD0000895E89409C097FB3EF490958095709521
:101AE00061957F4F8F4F9F4F9923A9F0F92F96E96A
:101AF000BB279395F695879577956795B795F111DF
:101B0000F8CFFAF4BB0F11F460FF1BC06F5F7F4F7B
:101B10008F4F9F4F16C0882311F096E911C077238D
:101B200021F09EE8872F762F05C0662371F096E896
:101B3000862F70E060E02AF09A95660F771F881F65
:101B4000DAF7880F9695879597F90895990F000809
:101B5000550FAA0BE0E8FEEF16161706E807F9077F
:101B6000C0F012161306E407F50798F0621B730B1A
:101B7000840B950B39F40A2661F0232B242B252B9B
:101B800021F408950A2609F4A140A6958FEF811D3E
:101B9000811D089597F99F6780E870E060E00895DF
:101BA0009FEF80EC089500240A9416161706180675
:101BB0000906089500240A94121613061406050651
:101BC0000895092E0394000C11F4882352F0BB0FE2
:101BD00040F4BF2B11F460FF04C06F5F7F4F8F4F45
:101BE0009F4F089557FD9058440F551F59F05F3F80
:101BF00071F04795880F97FB991F61F09F3F79F02F
:101C000087950895121613061406551FF2CF4695B0
:101C1000F1DF08C0161617061806991FF1CF869532
:101C20007105610508940895E894BB276627772716
:101C3000CB0197F908950E94A60D08F48FEF08953F
:101C40000E94330E0C94E10D0E94D30D38F00E94D7
:101C5000DA0D20F0952311F00C94CA0D0C94D00DE0
:101C600011240C94150E0E94F20D70F3959FC1F390
:101C7000950F50E0551F629FF001729FBB27F00D3A
:101C8000B11D639FAA27F00DB11DAA1F649F66278F
:101C9000B00DA11D661F829F2227B00DA11D621FDE
:101CA000739FB00DA11D621F839FA00D611D221F98
:101CB000749F3327A00D611D231F849F600D211D7C
:101CC000822F762F6A2F11249F5750409AF0F1F0FF
:101CD00088234AF0EE0FFF1FBB1F661F771F881F68
:101CE00091505040A9F79E3F510580F00C94CA0DC9
:101CF0000C94150E5F3FE4F3983ED4F386957795E8
:101D00006795B795F795E7959F5FC1F7FE2B880F0D
:101D1000911D9695879597F9089597FB072E16F4D0
:101D2000009407D077FD09D00E94A10E07FC05D0D2
:101D30003EF4909581959F4F0895709561957F4FE2
:101D40000895AA1BBB1B51E107C0AA1FBB1FA61702
:101D5000B70710F0A61BB70B881F991F5A95A9F754
:101D600080959095BC01CD010895EE0FFF1F059061
:0A1D7000F491E02D0994F894FFCFE0
:101D7A000000000000000000000000000000000059
:101D8A00000B00000000000000000000000000003E
:081D9A00000000090100000037
:00000001FF
